:100000000AC023C022C021C020C01FC01EC01DC006
:100010001CC01BC01AC011241FBECFEDCDBF10E005
:10002000A0E6B0E0EAE2F1E003C0C89531960D9297
:10003000A036B107D1F710E0A0E6B0E001C01D92F4
:10004000A236B107E1F717D06FC0DACFCF93DF93B5
:10005000CDB7DEB7E8E3F0E01082E7E3F0E080E15F
:100060008083E2E3F0E01082E1E3F0E08AE0808365
:10007000DF91CF910895CF93DF93CDB7DEB7A8E39B
:10008000B0E0E8E3F0E080818F7180628C93A7E3B9
:10009000B0E0E7E3F0E080818F7180628C9300C074
:1000A000E6E3F0E080819927807490700097C1F3B7
:1000B000A8E3B0E0E8E3F0E0808180618C9384EF16
:1000C00091E0909361008093600009C0809160008E
:1000D00090916100019790936100809360008091FE
:1000E000600090916100009789F7A8E3B0E0E8E331
:1000F000F0E090818FEE89238C9384EF91E09093D0
:1001000061008093600009C080916000909161005F
:1001100001979093610080936000809160009091BE
:0A0120006100009789F7BCCFFFCF04
:00000001FF
